Archive member included because of file (symbol)

c:/arm/arm/bin/../lib/gcc/arm-none-eabi/4.9.3/armv6-m\libgcc.a(_udivsi3.o)
                              ./system/src/stm32f0-stdperiph/stm32f0xx_rcc.o (__aeabi_uidiv)
c:/arm/arm/bin/../lib/gcc/arm-none-eabi/4.9.3/armv6-m\libgcc.a(_dvmd_tls.o)
                              c:/arm/arm/bin/../lib/gcc/arm-none-eabi/4.9.3/armv6-m\libgcc.a(_udivsi3.o) (__aeabi_idiv0)
c:/arm/arm/bin/../lib/gcc/arm-none-eabi/4.9.3/../../../../arm-none-eabi/lib/armv6-m\libg_nano.a(lib_a-errno.o)
                              ./system/src/newlib/_sbrk.o (__errno)
c:/arm/arm/bin/../lib/gcc/arm-none-eabi/4.9.3/../../../../arm-none-eabi/lib/armv6-m\libg_nano.a(lib_a-impure.o)
                              c:/arm/arm/bin/../lib/gcc/arm-none-eabi/4.9.3/../../../../arm-none-eabi/lib/armv6-m\libg_nano.a(lib_a-errno.o) (_impure_ptr)
c:/arm/arm/bin/../lib/gcc/arm-none-eabi/4.9.3/../../../../arm-none-eabi/lib/armv6-m\libg_nano.a(lib_a-strlen.o)
                              ./system/src/diag/Trace.o (strlen)
c:/arm/arm/bin/../lib/gcc/arm-none-eabi/4.9.3/../../../../arm-none-eabi/lib/armv6-m\libg_nano.a(lib_a-vsnprintf.o)
                              ./system/src/diag/Trace.o (vsnprintf)
c:/arm/arm/bin/../lib/gcc/arm-none-eabi/4.9.3/../../../../arm-none-eabi/lib/armv6-m\libg_nano.a(lib_a-nano-svfprintf.o)
                              c:/arm/arm/bin/../lib/gcc/arm-none-eabi/4.9.3/../../../../arm-none-eabi/lib/armv6-m\libg_nano.a(lib_a-vsnprintf.o) (_svfprintf_r)
c:/arm/arm/bin/../lib/gcc/arm-none-eabi/4.9.3/../../../../arm-none-eabi/lib/armv6-m\libg_nano.a(lib_a-nano-vfprintf_i.o)
                              c:/arm/arm/bin/../lib/gcc/arm-none-eabi/4.9.3/../../../../arm-none-eabi/lib/armv6-m\libg_nano.a(lib_a-nano-svfprintf.o) (_printf_i)
c:/arm/arm/bin/../lib/gcc/arm-none-eabi/4.9.3/../../../../arm-none-eabi/lib/armv6-m\libg_nano.a(lib_a-memchr.o)
                              c:/arm/arm/bin/../lib/gcc/arm-none-eabi/4.9.3/../../../../arm-none-eabi/lib/armv6-m\libg_nano.a(lib_a-nano-svfprintf.o) (memchr)
c:/arm/arm/bin/../lib/gcc/arm-none-eabi/4.9.3/../../../../arm-none-eabi/lib/armv6-m\libg_nano.a(lib_a-memcpy.o)
                              c:/arm/arm/bin/../lib/gcc/arm-none-eabi/4.9.3/../../../../arm-none-eabi/lib/armv6-m\libg_nano.a(lib_a-nano-svfprintf.o) (memcpy)
c:/arm/arm/bin/../lib/gcc/arm-none-eabi/4.9.3/../../../../arm-none-eabi/lib/armv6-m\libg_nano.a(lib_a-memmove.o)
                              c:/arm/arm/bin/../lib/gcc/arm-none-eabi/4.9.3/../../../../arm-none-eabi/lib/armv6-m\libg_nano.a(lib_a-nano-svfprintf.o) (memmove)
c:/arm/arm/bin/../lib/gcc/arm-none-eabi/4.9.3/../../../../arm-none-eabi/lib/armv6-m\libg_nano.a(lib_a-nano-freer.o)
                              c:/arm/arm/bin/../lib/gcc/arm-none-eabi/4.9.3/../../../../arm-none-eabi/lib/armv6-m\libg_nano.a(lib_a-nano-svfprintf.o) (_free_r)
c:/arm/arm/bin/../lib/gcc/arm-none-eabi/4.9.3/../../../../arm-none-eabi/lib/armv6-m\libg_nano.a(lib_a-nano-mallocr.o)
                              c:/arm/arm/bin/../lib/gcc/arm-none-eabi/4.9.3/../../../../arm-none-eabi/lib/armv6-m\libg_nano.a(lib_a-nano-svfprintf.o) (_malloc_r)
c:/arm/arm/bin/../lib/gcc/arm-none-eabi/4.9.3/../../../../arm-none-eabi/lib/armv6-m\libg_nano.a(lib_a-nano-reallocr.o)
                              c:/arm/arm/bin/../lib/gcc/arm-none-eabi/4.9.3/../../../../arm-none-eabi/lib/armv6-m\libg_nano.a(lib_a-nano-svfprintf.o) (_realloc_r)
c:/arm/arm/bin/../lib/gcc/arm-none-eabi/4.9.3/../../../../arm-none-eabi/lib/armv6-m\libg_nano.a(lib_a-sbrkr.o)
                              c:/arm/arm/bin/../lib/gcc/arm-none-eabi/4.9.3/../../../../arm-none-eabi/lib/armv6-m\libg_nano.a(lib_a-nano-mallocr.o) (_sbrk_r)
c:/arm/arm/bin/../lib/gcc/arm-none-eabi/4.9.3/../../../../arm-none-eabi/lib/armv6-m\libg_nano.a(lib_a-nano-msizer.o)
                              c:/arm/arm/bin/../lib/gcc/arm-none-eabi/4.9.3/../../../../arm-none-eabi/lib/armv6-m\libg_nano.a(lib_a-nano-reallocr.o) (_malloc_usable_size_r)

Allocating common symbols
Common symbol       size              file

errno               0x4               ./system/src/newlib/_syscalls.o

Discarded input sections

 .group         0x00000000        0x8 ./system/src/stm32f0-stdperiph/stm32f0xx_exti.o
 .group         0x00000000        0x8 ./system/src/stm32f0-stdperiph/stm32f0xx_exti.o
 .group         0x00000000        0x8 ./system/src/stm32f0-stdperiph/stm32f0xx_exti.o
 .group         0x00000000        0x8 ./system/src/stm32f0-stdperiph/stm32f0xx_exti.o
 .group         0x00000000        0x8 ./system/src/stm32f0-stdperiph/stm32f0xx_exti.o
 .group         0x00000000        0x8 ./system/src/stm32f0-stdperiph/stm32f0xx_exti.o
 .group         0x00000000        0x8 ./system/src/stm32f0-stdperiph/stm32f0xx_exti.o
 .group         0x00000000        0x8 ./system/src/stm32f0-stdperiph/stm32f0xx_exti.o
 .group         0x00000000        0x8 ./system/src/stm32f0-stdperiph/stm32f0xx_exti.o
 .group         0x00000000        0x8 ./system/src/stm32f0-stdperiph/stm32f0xx_exti.o
 .group         0x00000000        0x8 ./system/src/stm32f0-stdperiph/stm32f0xx_exti.o
 .group         0x00000000        0x8 ./system/src/stm32f0-stdperiph/stm32f0xx_exti.o
 .group         0x00000000        0x8 ./system/src/stm32f0-stdperiph/stm32f0xx_exti.o
 .group         0x00000000        0x8 ./system/src/stm32f0-stdperiph/stm32f0xx_exti.o
 .group         0x00000000        0x8 ./system/src/stm32f0-stdperiph/stm32f0xx_exti.o
 .group         0x00000000        0x8 ./system/src/stm32f0-stdperiph/stm32f0xx_exti.o
 .group         0x00000000        0x8 ./system/src/stm32f0-stdperiph/stm32f0xx_exti.o
 .group         0x00000000        0x8 ./system/src/stm32f0-stdperiph/stm32f0xx_exti.o
Memory Configuration

Name             Origin             Length             Attributes
RAM              0x20000000         0x00001000         xrw
CCMRAM           0x00000000         0x00000000         xrw
FLASH            0x08000000         0x00004000         xr
FLASHB1          0x00000000         0x00000000         xr
EXTMEMB0         0x00000000         0x00000000         xr
EXTMEMB1         0x00000000         0x00000000         xr
EXTMEMB2         0x00000000         0x00000000         xr
EXTMEMB3         0x00000000         0x00000000         xr
MEMORY_ARRAY     0x00000000         0x00000000         xrw
*default*        0x00000000         0xffffffff

Linker script and memory map

LOAD ./system/src/stm32f0-stdperiph/stm32f0xx_exti.o
LOAD ./system/src/stm32f0-stdperiph/stm32f0xx_gpio.o
LOAD ./system/src/stm32f0-stdperiph/stm32f0xx_misc.o
LOAD ./system/src/stm32f0-stdperiph/stm32f0xx_rcc.o
LOAD ./system/src/stm32f0-stdperiph/stm32f0xx_syscfg.o
LOAD ./system/src/newlib/_cxx.o
LOAD ./system/src/newlib/_exit.o
LOAD ./system/src/newlib/_sbrk.o
LOAD ./system/src/newlib/_startup.o
LOAD ./system/src/newlib/_syscalls.o
LOAD ./system/src/newlib/assert.o
LOAD ./system/src/diag/Trace.o
LOAD ./system/src/diag/trace_impl.o
LOAD ./system/src/cortexm/_initialize_hardware.o
LOAD ./system/src/cortexm/_reset_hardware.o
LOAD ./system/src/cortexm/exception_handlers.o
LOAD ./system/src/cmsis/system_stm32f0xx.o
LOAD ./system/src/cmsis/vectors_stm32f0xx.o
LOAD ./src/_write.o
LOAD ./src/main.o
LOAD ./src/stm32f0xx_it.o
LOAD c:/arm/arm/bin/../lib/gcc/arm-none-eabi/4.9.3/../../../../arm-none-eabi/lib/armv6-m\libstdc++_nano.a
LOAD c:/arm/arm/bin/../lib/gcc/arm-none-eabi/4.9.3/../../../../arm-none-eabi/lib/armv6-m\libm.a
START GROUP
LOAD c:/arm/arm/bin/../lib/gcc/arm-none-eabi/4.9.3/armv6-m\libgcc.a
LOAD c:/arm/arm/bin/../lib/gcc/arm-none-eabi/4.9.3/../../../../arm-none-eabi/lib/armv6-m\libg_nano.a
LOAD c:/arm/arm/bin/../lib/gcc/arm-none-eabi/4.9.3/../../../../arm-none-eabi/lib/armv6-m\libc_nano.a
END GROUP
START GROUP
LOAD c:/arm/arm/bin/../lib/gcc/arm-none-eabi/4.9.3/armv6-m\libgcc.a
LOAD c:/arm/arm/bin/../lib/gcc/arm-none-eabi/4.9.3/../../../../arm-none-eabi/lib/armv6-m\libc_nano.a
END GROUP
                0x20001000                __stack = (ORIGIN (RAM) + 0x1000)
                0x20001000                _estack = __stack
                0x00000400                __Main_Stack_Size = 0x400
                0x00000400                PROVIDE (_Main_Stack_Size, __Main_Stack_Size)
                0x20000c00                __Main_Stack_Limit = (__stack - __Main_Stack_Size)
                0x20000c00                PROVIDE (_Main_Stack_Limit, __Main_Stack_Limit)
                0x00000100                _Minimum_Stack_Size = 0x100
                0x20000128                PROVIDE (_Heap_Begin, _end_noinit)
                0x20000c00                PROVIDE (_Heap_Limit, (__stack - __Main_Stack_Size))

.isr_vector     0x08000000      0x230
                0x08000000                . = ALIGN (0x4)
 *(.isr_vector)
 .isr_vector    0x08000000       0xc4 ./system/src/cmsis/vectors_stm32f0xx.o
                0x08000000                g_pfnVectors
 *(.cfmconfig)
 *(.after_vectors .after_vectors.*)
 .after_vectors
                0x080000c4      0x118 ./system/src/newlib/_startup.o
                0x080000c4                _start
 .after_vectors
                0x080001dc       0x50 ./system/src/cortexm/exception_handlers.o
                0x080001dc                Reset_Handler
                0x080001e4                NMI_Handler
                0x080001e8                HardFault_Handler
                0x08000200                HardFault_Handler_C
                0x0800021c                SVC_Handler
                0x08000220                PendSV_Handler
                0x08000224                SysTick_Handler
 .after_vectors
                0x0800022c        0x4 ./system/src/cmsis/vectors_stm32f0xx.o
                0x0800022c                TIM1_CC_IRQHandler
                0x0800022c                TSC_IRQHandler
                0x0800022c                ADC1_COMP_IRQHandler
                0x0800022c                PVD_IRQHandler
                0x0800022c                I2C1_IRQHandler
                0x0800022c                RCC_CRS_IRQHandler
                0x0800022c                SPI1_IRQHandler
                0x0800022c                TIM6_DAC_IRQHandler
                0x0800022c                USART3_4_IRQHandler
                0x0800022c                EXTI2_3_IRQHandler
                0x0800022c                ADC1_IRQHandler
                0x0800022c                I2C2_IRQHandler
                0x0800022c                TIM17_IRQHandler
                0x0800022c                CEC_CAN_IRQHandler
                0x0800022c                RTC_IRQHandler
                0x0800022c                PVD_VDDIO2_IRQHandler
                0x0800022c                DMA1_Channel4_5_6_7_IRQHandler
                0x0800022c                TIM16_IRQHandler
                0x0800022c                TIM3_IRQHandler
                0x0800022c                EXTI4_15_IRQHandler
                0x0800022c                RCC_IRQHandler
                0x0800022c                DMA1_Channel1_IRQHandler
                0x0800022c                Default_Handler
                0x0800022c                CEC_IRQHandler
                0x0800022c                TIM14_IRQHandler
                0x0800022c                DMA1_Channel4_5_IRQHandler
                0x0800022c                TIM7_IRQHandler
                0x0800022c                TIM15_IRQHandler
                0x0800022c                USB_IRQHandler
                0x0800022c                SPI2_IRQHandler
                0x0800022c                TS_IRQHandler
                0x0800022c                WWDG_IRQHandler
                0x0800022c                TIM2_IRQHandler
                0x0800022c                DMA1_Channel2_3_IRQHandler
                0x0800022c                USART2_IRQHandler
                0x0800022c                FLASH_IRQHandler
                0x0800022c                USART1_IRQHandler
                0x0800022c                TIM1_BRK_UP_TRG_COM_IRQHandler
                0x08000230                . = ALIGN (0x4)

.inits          0x08000230        0x0
                0x08000230                . = ALIGN (0x4)
 *(.init)
 *(.fini)
                0x08000230                . = ALIGN (0x4)
                0x08000230                PROVIDE (__preinit_array_start, .)
 *(.preinit_array_sysinit .preinit_array_sysinit.*)
 *(.preinit_array_platform .preinit_array_platform.*)
 *(.preinit_array .preinit_array.*)
                0x08000230                PROVIDE (__preinit_array_end, .)
                0x08000230                . = ALIGN (0x4)
                0x08000230                PROVIDE (__init_array_start, .)
 *(SORT(.init_array.*))
 *(.init_array)
                0x08000230                PROVIDE (__init_array_end, .)
                0x08000230                . = ALIGN (0x4)
                0x08000230                PROVIDE (__fini_array_start, .)
 *(SORT(.fini_array.*))
 *(.fini_array)
                0x08000230                PROVIDE (__fini_array_end, .)
                0x08000230                . = ALIGN (0x4)

.flashtext      0x08000230        0x0
                0x08000230                . = ALIGN (0x4)
 *(.flashtext .flashtext.*)
                0x08000230                . = ALIGN (0x4)

.text           0x08000230     0x15d1
                0x08000230                . = ALIGN (0x4)
 *(.text .text.*)
 .text.EXTI_Init
                0x08000230       0xcc ./system/src/stm32f0-stdperiph/stm32f0xx_exti.o
                0x08000230                EXTI_Init
 .text.EXTI_GetITStatus
                0x080002fc       0xe4 ./system/src/stm32f0-stdperiph/stm32f0xx_exti.o
                0x080002fc                EXTI_GetITStatus
 .text.EXTI_ClearITPendingBit
                0x080003e0       0x28 ./system/src/stm32f0-stdperiph/stm32f0xx_exti.o
                0x080003e0                EXTI_ClearITPendingBit
 .text.GPIO_Init
                0x08000408      0x11c ./system/src/stm32f0-stdperiph/stm32f0xx_gpio.o
                0x08000408                GPIO_Init
 .text.GPIO_ReadInputDataBit
                0x08000524       0xc8 ./system/src/stm32f0-stdperiph/stm32f0xx_gpio.o
                0x08000524                GPIO_ReadInputDataBit
 .text.GPIO_SetBits
                0x080005ec       0x60 ./system/src/stm32f0-stdperiph/stm32f0xx_gpio.o
                0x080005ec                GPIO_SetBits
 .text.GPIO_ResetBits
                0x0800064c       0x60 ./system/src/stm32f0-stdperiph/stm32f0xx_gpio.o
                0x0800064c                GPIO_ResetBits
 .text.NVIC_Init
                0x080006ac       0x78 ./system/src/stm32f0-stdperiph/stm32f0xx_misc.o
                0x080006ac                NVIC_Init
 .text.RCC_AHBPeriphClockCmd
                0x08000724       0x50 ./system/src/stm32f0-stdperiph/stm32f0xx_rcc.o
                0x08000724                RCC_AHBPeriphClockCmd
 .text.SYSCFG_EXTILineConfig
                0x08000774       0x48 ./system/src/stm32f0-stdperiph/stm32f0xx_syscfg.o
                0x08000774                SYSCFG_EXTILineConfig
 .text._exit    0x080007bc        0x4 ./system/src/newlib/_exit.o
                0x080007bc                _exit
 .text.abort    0x080007c0       0x14 ./system/src/newlib/_exit.o
                0x080007c0                abort
 .text._sbrk    0x080007d4       0x44 ./system/src/newlib/_sbrk.o
                0x080007d4                _sbrk
 .text.__initialize_args
                0x08000818       0x10 ./system/src/newlib/_syscalls.o
                0x08000818                __initialize_args
 .text.assert_failed
                0x08000828       0x18 ./system/src/newlib/assert.o
                0x08000828                assert_failed
 .text.trace_printf
                0x08000840       0x30 ./system/src/diag/Trace.o
                0x08000840                trace_printf
 .text.trace_puts
                0x08000870       0x20 ./system/src/diag/Trace.o
                0x08000870                trace_puts
 .text.trace_write
                0x08000890        0x8 ./system/src/diag/trace_impl.o
                0x08000890                trace_write
 .text.__initialize_hardware_early
                0x08000898        0x8 ./system/src/cortexm/_initialize_hardware.o
                0x08000898                __initialize_hardware_early
 .text.__initialize_hardware
                0x080008a0        0x8 ./system/src/cortexm/_initialize_hardware.o
                0x080008a0                __initialize_hardware
 .text.dumpExceptionStack
                0x080008a8       0x88 ./system/src/cortexm/exception_handlers.o
                0x080008a8                dumpExceptionStack
 .text.SetSysClock
                0x08000930       0xb0 ./system/src/cmsis/system_stm32f0xx.o
 .text.SystemInit
                0x080009e0       0x64 ./system/src/cmsis/system_stm32f0xx.o
                0x080009e0                SystemInit
 .text.SystemCoreClockUpdate
                0x08000a44       0x90 ./system/src/cmsis/system_stm32f0xx.o
                0x08000a44                SystemCoreClockUpdate
 .text.main     0x08000ad4       0x7c ./src/main.o
                0x08000ad4                main
 .text.EXTI0_1_IRQHandler
                0x08000b50       0x90 ./src/stm32f0xx_it.o
                0x08000b50                EXTI0_1_IRQHandler
 .text          0x08000be0      0x120 c:/arm/arm/bin/../lib/gcc/arm-none-eabi/4.9.3/armv6-m\libgcc.a(_udivsi3.o)
                0x08000be0                __aeabi_uidiv
                0x08000be0                __udivsi3
                0x08000cec                __aeabi_uidivmod
 .text          0x08000d00        0x4 c:/arm/arm/bin/../lib/gcc/arm-none-eabi/4.9.3/armv6-m\libgcc.a(_dvmd_tls.o)
                0x08000d00                __aeabi_idiv0
                0x08000d00                __aeabi_ldiv0
 .text.__errno  0x08000d04        0xc c:/arm/arm/bin/../lib/gcc/arm-none-eabi/4.9.3/../../../../arm-none-eabi/lib/armv6-m\libg_nano.a(lib_a-errno.o)
                0x08000d04                __errno
 .text.strlen   0x08000d10        0xe c:/arm/arm/bin/../lib/gcc/arm-none-eabi/4.9.3/../../../../arm-none-eabi/lib/armv6-m\libg_nano.a(lib_a-strlen.o)
                0x08000d10                strlen
 .text._vsnprintf_r
                0x08000d1e       0x54 c:/arm/arm/bin/../lib/gcc/arm-none-eabi/4.9.3/../../../../arm-none-eabi/lib/armv6-m\libg_nano.a(lib_a-vsnprintf.o)
                0x08000d1e                _vsniprintf_r
                0x08000d1e                _vsnprintf_r
 *fill*         0x08000d72        0x2 
 .text.vsnprintf
                0x08000d74       0x20 c:/arm/arm/bin/../lib/gcc/arm-none-eabi/4.9.3/../../../../arm-none-eabi/lib/armv6-m\libg_nano.a(lib_a-vsnprintf.o)
                0x08000d74                vsniprintf
                0x08000d74                vsnprintf
 .text.__ssputs_r
                0x08000d94       0xc0 c:/arm/arm/bin/../lib/gcc/arm-none-eabi/4.9.3/../../../../arm-none-eabi/lib/armv6-m\libg_nano.a(lib_a-nano-svfprintf.o)
                0x08000d94                __ssputs_r
 .text._svfprintf_r
                0x08000e54      0x1ec c:/arm/arm/bin/../lib/gcc/arm-none-eabi/4.9.3/../../../../arm-none-eabi/lib/armv6-m\libg_nano.a(lib_a-nano-svfprintf.o)
                0x08000e54                _svfiprintf_r
                0x08000e54                _svfprintf_r
 .text._printf_common
                0x08001040       0xdc c:/arm/arm/bin/../lib/gcc/arm-none-eabi/4.9.3/../../../../arm-none-eabi/lib/armv6-m\libg_nano.a(lib_a-nano-vfprintf_i.o)
                0x08001040                _printf_common
 .text._printf_i
                0x0800111c      0x230 c:/arm/arm/bin/../lib/gcc/arm-none-eabi/4.9.3/../../../../arm-none-eabi/lib/armv6-m\libg_nano.a(lib_a-nano-vfprintf_i.o)
                0x0800111c                _printf_i
 .text.memchr   0x0800134c       0x16 c:/arm/arm/bin/../lib/gcc/arm-none-eabi/4.9.3/../../../../arm-none-eabi/lib/armv6-m\libg_nano.a(lib_a-memchr.o)
                0x0800134c                memchr
 .text.memcpy   0x08001362       0x12 c:/arm/arm/bin/../lib/gcc/arm-none-eabi/4.9.3/../../../../arm-none-eabi/lib/armv6-m\libg_nano.a(lib_a-memcpy.o)
                0x08001362                memcpy
 .text.memmove  0x08001374       0x28 c:/arm/arm/bin/../lib/gcc/arm-none-eabi/4.9.3/../../../../arm-none-eabi/lib/armv6-m\libg_nano.a(lib_a-memmove.o)
                0x08001374                memmove
 .text._free_r  0x0800139c       0x8c c:/arm/arm/bin/../lib/gcc/arm-none-eabi/4.9.3/../../../../arm-none-eabi/lib/armv6-m\libg_nano.a(lib_a-nano-freer.o)
                0x0800139c                _free_r
 .text._malloc_r
                0x08001428       0xb0 c:/arm/arm/bin/../lib/gcc/arm-none-eabi/4.9.3/../../../../arm-none-eabi/lib/armv6-m\libg_nano.a(lib_a-nano-mallocr.o)
                0x08001428                _malloc_r
 .text._realloc_r
                0x080014d8       0x4c c:/arm/arm/bin/../lib/gcc/arm-none-eabi/4.9.3/../../../../arm-none-eabi/lib/armv6-m\libg_nano.a(lib_a-nano-reallocr.o)
                0x080014d8                _realloc_r
 .text._sbrk_r  0x08001524       0x24 c:/arm/arm/bin/../lib/gcc/arm-none-eabi/4.9.3/../../../../arm-none-eabi/lib/armv6-m\libg_nano.a(lib_a-sbrkr.o)
                0x08001524                _sbrk_r
 .text._malloc_usable_size_r
                0x08001548       0x16 c:/arm/arm/bin/../lib/gcc/arm-none-eabi/4.9.3/../../../../arm-none-eabi/lib/armv6-m\libg_nano.a(lib_a-nano-msizer.o)
                0x08001548                _malloc_usable_size_r
 *(.rodata .rodata.*)
 *fill*         0x0800155e        0x2 
 .rodata.str1.4
                0x08001560       0x31 ./system/src/stm32f0-stdperiph/stm32f0xx_exti.o
                                 0x34 (size before relaxing)
 *fill*         0x08001591        0x3 
 .rodata.str1.4
                0x08001594       0x31 ./system/src/stm32f0-stdperiph/stm32f0xx_gpio.o
                                 0x34 (size before relaxing)
 *fill*         0x080015c5        0x3 
 .rodata.str1.4
                0x080015c8       0x31 ./system/src/stm32f0-stdperiph/stm32f0xx_misc.o
                                 0x34 (size before relaxing)
 *fill*         0x080015f9        0x3 
 .rodata.str1.4
                0x080015fc       0x30 ./system/src/stm32f0-stdperiph/stm32f0xx_rcc.o
 .rodata.str1.4
                0x0800162c       0x33 ./system/src/stm32f0-stdperiph/stm32f0xx_syscfg.o
                                 0x34 (size before relaxing)
 *fill*         0x0800165f        0x1 
 .rodata.str1.4
                0x08001660       0x14 ./system/src/newlib/_exit.o
 .rodata.str1.4
                0x08001674       0x6b ./system/src/newlib/assert.o
                                 0x70 (size before relaxing)
 *fill*         0x080016df        0x1 
 .rodata.str1.4
                0x080016e0       0x29 ./system/src/diag/Trace.o
                                 0x30 (size before relaxing)
 *fill*         0x08001709        0x3 
 .rodata.str1.4
                0x0800170c       0xc0 ./system/src/cortexm/exception_handlers.o
 .rodata.str1.1
                0x080017cc        0x2 c:/arm/arm/bin/../lib/gcc/arm-none-eabi/4.9.3/../../../../arm-none-eabi/lib/armv6-m\libg_nano.a(lib_a-impure.o)
 .rodata.str1.1
                0x080017ce       0x11 c:/arm/arm/bin/../lib/gcc/arm-none-eabi/4.9.3/../../../../arm-none-eabi/lib/armv6-m\libg_nano.a(lib_a-nano-svfprintf.o)
 .rodata.str1.1
                0x080017df       0x22 c:/arm/arm/bin/../lib/gcc/arm-none-eabi/4.9.3/../../../../arm-none-eabi/lib/armv6-m\libg_nano.a(lib_a-nano-vfprintf_i.o)
 *(vtable)
 *(.eh_frame*)
 *(.glue_7)
 .glue_7        0x00000000        0x0 linker stubs
 *(.glue_7t)
 .glue_7t       0x00000000        0x0 linker stubs

.vfp11_veneer   0x08001804        0x0
 .vfp11_veneer  0x00000000        0x0 linker stubs

.v4_bx          0x08001804        0x0
 .v4_bx         0x00000000        0x0 linker stubs

.iplt           0x08001804        0x0
 .iplt          0x00000000        0x0 ./system/src/stm32f0-stdperiph/stm32f0xx_exti.o

.rel.dyn        0x08001804        0x0
 .rel.iplt      0x00000000        0x0 ./system/src/stm32f0-stdperiph/stm32f0xx_exti.o

.ARM.extab
 *(.ARM.extab* .gnu.linkonce.armextab.*)
                0x08001804                __exidx_start = .

.ARM.exidx
 *(.ARM.exidx* .gnu.linkonce.armexidx.*)
                0x08001804                __exidx_end = .
                0x08001804                . = ALIGN (0x4)
                0x08001804                _etext = .
                0x08001804                __etext = .
                0x08001804                _sidata = _etext

.data           0x20000000       0x88 load address 0x08001804
                0x20000000                . = ALIGN (0x4)
                0x20000000                _sdata = .
                0x20000000                __data_start__ = .
 *(.data_begin .data_begin.*)
 .data_begin    0x20000000        0x4 ./system/src/newlib/_startup.o
 *(.data .data.*)
 .data.argv.4062
                0x20000004        0x8 ./system/src/newlib/_syscalls.o
 .data.AHBPrescTable
                0x2000000c       0x10 ./system/src/cmsis/system_stm32f0xx.o
                0x2000000c                AHBPrescTable
 .data.SystemCoreClock
                0x2000001c        0x4 ./system/src/cmsis/system_stm32f0xx.o
                0x2000001c                SystemCoreClock
 .data.impure_data
                0x20000020       0x60 c:/arm/arm/bin/../lib/gcc/arm-none-eabi/4.9.3/../../../../arm-none-eabi/lib/armv6-m\libg_nano.a(lib_a-impure.o)
 .data._impure_ptr
                0x20000080        0x4 c:/arm/arm/bin/../lib/gcc/arm-none-eabi/4.9.3/../../../../arm-none-eabi/lib/armv6-m\libg_nano.a(lib_a-impure.o)
                0x20000080                _impure_ptr
 *(.data_end .data_end.*)
 .data_end      0x20000084        0x4 ./system/src/newlib/_startup.o
                0x20000088                . = ALIGN (0x4)
                0x20000088                _edata = .
                0x20000088                __data_end__ = .

.igot.plt       0x20000088        0x0 load address 0x0800188c
 .igot.plt      0x00000000        0x0 ./system/src/stm32f0-stdperiph/stm32f0xx_exti.o

.bss            0x20000088       0xa0 load address 0x0800188c
                0x20000088                . = ALIGN (0x4)
                0x20000088                __bss_start__ = .
                0x20000088                _sbss = .
 *(.bss_begin .bss_begin.*)
 .bss_begin     0x20000088        0x4 ./system/src/newlib/_startup.o
 *(.bss .bss.*)
 .bss.current_heap_end.3856
                0x2000008c        0x4 ./system/src/newlib/_sbrk.o
 .bss.name.4061
                0x20000090        0x4 ./system/src/newlib/_syscalls.o
 .bss.buf.4992  0x20000094       0x80 ./system/src/diag/Trace.o
 .bss.count     0x20000114        0x2 ./src/stm32f0xx_it.o
                0x20000114                count
 *fill*         0x20000116        0x2 
 .bss.__malloc_sbrk_start
                0x20000118        0x4 c:/arm/arm/bin/../lib/gcc/arm-none-eabi/4.9.3/../../../../arm-none-eabi/lib/armv6-m\libg_nano.a(lib_a-nano-mallocr.o)
                0x20000118                __malloc_sbrk_start
 .bss.__malloc_free_list
                0x2000011c        0x4 c:/arm/arm/bin/../lib/gcc/arm-none-eabi/4.9.3/../../../../arm-none-eabi/lib/armv6-m\libg_nano.a(lib_a-nano-mallocr.o)
                0x2000011c                __malloc_free_list
 *(COMMON)
 COMMON         0x20000120        0x4 ./system/src/newlib/_syscalls.o
                0x20000120                errno
 *(.bss_end .bss_end.*)
 .bss_end       0x20000124        0x4 ./system/src/newlib/_startup.o
                0x20000128                . = ALIGN (0x4)
                0x20000128                __bss_end__ = .
                0x20000128                _ebss = .

.noinit         0x20000128        0x0
                0x20000128                . = ALIGN (0x4)
                0x20000128                _noinit = .
 *(.noinit .noinit.*)
                0x20000128                . = ALIGN (0x4)
                0x20000128                _end_noinit = .
                0x20000128                PROVIDE (end, _end_noinit)
                0x20000128                PROVIDE (_end, _end_noinit)
                0x20000128                PROVIDE (__end, _end_noinit)
                0x20000128                PROVIDE (__end__, _end_noinit)

._check_stack   0x20000128      0x100 load address 0x0800192c
                0x20000128                . = ALIGN (0x4)
                0x20000228                . = (. + _Minimum_Stack_Size)
 *fill*         0x20000128      0x100 
                0x20000228                . = ALIGN (0x4)

.bss_CCMRAM
 *(.bss.CCMRAM .bss.CCMRAM.*)

.b1text
 *(.b1text)
 *(.b1rodata)
 *(.b1rodata.*)

.eb0text
 *(.eb0text)
 *(.eb0rodata)
 *(.eb0rodata.*)

.eb1text
 *(.eb1text)
 *(.eb1rodata)
 *(.eb1rodata.*)

.eb2text
 *(.eb2text)
 *(.eb2rodata)
 *(.eb2rodata.*)

.eb3text
 *(.eb3text)
 *(.eb3rodata)
 *(.eb3rodata.*)

.stab
 *(.stab)

.stabstr
 *(.stabstr)

.stab.excl
 *(.stab.excl)

.stab.exclstr
 *(.stab.exclstr)

.stab.index
 *(.stab.index)

.stab.indexstr
 *(.stab.indexstr)

.comment        0x00000000       0x70
 *(.comment)
 .comment       0x00000000       0x70 ./system/src/stm32f0-stdperiph/stm32f0xx_exti.o
                                 0x71 (size before relaxing)
 .comment       0x00000000       0x71 ./system/src/stm32f0-stdperiph/stm32f0xx_gpio.o
 .comment       0x00000000       0x71 ./system/src/stm32f0-stdperiph/stm32f0xx_misc.o
 .comment       0x00000000       0x71 ./system/src/stm32f0-stdperiph/stm32f0xx_rcc.o
 .comment       0x00000000       0x71 ./system/src/stm32f0-stdperiph/stm32f0xx_syscfg.o
 .comment       0x00000000       0x71 ./system/src/newlib/_exit.o
 .comment       0x00000000       0x71 ./system/src/newlib/_sbrk.o
 .comment       0x00000000       0x71 ./system/src/newlib/_startup.o
 .comment       0x00000000       0x71 ./system/src/newlib/_syscalls.o
 .comment       0x00000000       0x71 ./system/src/newlib/assert.o
 .comment       0x00000000       0x71 ./system/src/diag/Trace.o
 .comment       0x00000000       0x71 ./system/src/diag/trace_impl.o
 .comment       0x00000000       0x71 ./system/src/cortexm/_initialize_hardware.o
 .comment       0x00000000       0x71 ./system/src/cortexm/exception_handlers.o
 .comment       0x00000000       0x71 ./system/src/cmsis/system_stm32f0xx.o
 .comment       0x00000000       0x71 ./system/src/cmsis/vectors_stm32f0xx.o
 .comment       0x00000000       0x71 ./src/main.o
 .comment       0x00000000       0x71 ./src/stm32f0xx_it.o

.ARM.attributes
                0x00000000       0x31
 .ARM.attributes
                0x00000000       0x31 ./system/src/stm32f0-stdperiph/stm32f0xx_exti.o
 .ARM.attributes
                0x00000031       0x31 ./system/src/stm32f0-stdperiph/stm32f0xx_gpio.o
 .ARM.attributes
                0x00000062       0x31 ./system/src/stm32f0-stdperiph/stm32f0xx_misc.o
 .ARM.attributes
                0x00000093       0x31 ./system/src/stm32f0-stdperiph/stm32f0xx_rcc.o
 .ARM.attributes
                0x000000c4       0x31 ./system/src/stm32f0-stdperiph/stm32f0xx_syscfg.o
 .ARM.attributes
                0x000000f5       0x31 ./system/src/newlib/_exit.o
 .ARM.attributes
                0x00000126       0x31 ./system/src/newlib/_sbrk.o
 .ARM.attributes
                0x00000157       0x31 ./system/src/newlib/_startup.o
 .ARM.attributes
                0x00000188       0x31 ./system/src/newlib/_syscalls.o
 .ARM.attributes
                0x000001b9       0x31 ./system/src/newlib/assert.o
 .ARM.attributes
                0x000001ea       0x31 ./system/src/diag/Trace.o
 .ARM.attributes
                0x0000021b       0x31 ./system/src/diag/trace_impl.o
 .ARM.attributes
                0x0000024c       0x31 ./system/src/cortexm/_initialize_hardware.o
 .ARM.attributes
                0x0000027d       0x31 ./system/src/cortexm/exception_handlers.o
 .ARM.attributes
                0x000002ae       0x31 ./system/src/cmsis/system_stm32f0xx.o
 .ARM.attributes
                0x000002df       0x31 ./system/src/cmsis/vectors_stm32f0xx.o
 .ARM.attributes
                0x00000310       0x31 ./src/main.o
 .ARM.attributes
                0x00000341       0x31 ./src/stm32f0xx_it.o
 .ARM.attributes
                0x00000372       0x1e c:/arm/arm/bin/../lib/gcc/arm-none-eabi/4.9.3/armv6-m\libgcc.a(_udivsi3.o)
 .ARM.attributes
                0x00000390       0x1e c:/arm/arm/bin/../lib/gcc/arm-none-eabi/4.9.3/armv6-m\libgcc.a(_dvmd_tls.o)
 .ARM.attributes
                0x000003ae       0x2c c:/arm/arm/bin/../lib/gcc/arm-none-eabi/4.9.3/../../../../arm-none-eabi/lib/armv6-m\libg_nano.a(lib_a-errno.o)
 .ARM.attributes
                0x000003da       0x2c c:/arm/arm/bin/../lib/gcc/arm-none-eabi/4.9.3/../../../../arm-none-eabi/lib/armv6-m\libg_nano.a(lib_a-impure.o)
 .ARM.attributes
                0x00000406       0x2c c:/arm/arm/bin/../lib/gcc/arm-none-eabi/4.9.3/../../../../arm-none-eabi/lib/armv6-m\libg_nano.a(lib_a-strlen.o)
 .ARM.attributes
                0x00000432       0x2c c:/arm/arm/bin/../lib/gcc/arm-none-eabi/4.9.3/../../../../arm-none-eabi/lib/armv6-m\libg_nano.a(lib_a-vsnprintf.o)
 .ARM.attributes
                0x0000045e       0x2c c:/arm/arm/bin/../lib/gcc/arm-none-eabi/4.9.3/../../../../arm-none-eabi/lib/armv6-m\libg_nano.a(lib_a-nano-svfprintf.o)
 .ARM.attributes
                0x0000048a       0x2c c:/arm/arm/bin/../lib/gcc/arm-none-eabi/4.9.3/../../../../arm-none-eabi/lib/armv6-m\libg_nano.a(lib_a-nano-vfprintf_i.o)
 .ARM.attributes
                0x000004b6       0x2c c:/arm/arm/bin/../lib/gcc/arm-none-eabi/4.9.3/../../../../arm-none-eabi/lib/armv6-m\libg_nano.a(lib_a-memchr.o)
 .ARM.attributes
                0x000004e2       0x2c c:/arm/arm/bin/../lib/gcc/arm-none-eabi/4.9.3/../../../../arm-none-eabi/lib/armv6-m\libg_nano.a(lib_a-memcpy.o)
 .ARM.attributes
                0x0000050e       0x2c c:/arm/arm/bin/../lib/gcc/arm-none-eabi/4.9.3/../../../../arm-none-eabi/lib/armv6-m\libg_nano.a(lib_a-memmove.o)
 .ARM.attributes
                0x0000053a       0x2c c:/arm/arm/bin/../lib/gcc/arm-none-eabi/4.9.3/../../../../arm-none-eabi/lib/armv6-m\libg_nano.a(lib_a-nano-freer.o)
 .ARM.attributes
                0x00000566       0x2c c:/arm/arm/bin/../lib/gcc/arm-none-eabi/4.9.3/../../../../arm-none-eabi/lib/armv6-m\libg_nano.a(lib_a-nano-mallocr.o)
 .ARM.attributes
                0x00000592       0x2c c:/arm/arm/bin/../lib/gcc/arm-none-eabi/4.9.3/../../../../arm-none-eabi/lib/armv6-m\libg_nano.a(lib_a-nano-reallocr.o)
 .ARM.attributes
                0x000005be       0x2c c:/arm/arm/bin/../lib/gcc/arm-none-eabi/4.9.3/../../../../arm-none-eabi/lib/armv6-m\libg_nano.a(lib_a-sbrkr.o)
 .ARM.attributes
                0x000005ea       0x2c c:/arm/arm/bin/../lib/gcc/arm-none-eabi/4.9.3/../../../../arm-none-eabi/lib/armv6-m\libg_nano.a(lib_a-nano-msizer.o)

.debug
 *(.debug)

.line
 *(.line)

.debug_srcinfo
 *(.debug_srcinfo)

.debug_sfnames
 *(.debug_sfnames)

.debug_aranges  0x00000000      0x510
 *(.debug_aranges)
 .debug_aranges
                0x00000000       0x58 ./system/src/stm32f0-stdperiph/stm32f0xx_exti.o
 .debug_aranges
                0x00000058       0x80 ./system/src/stm32f0-stdperiph/stm32f0xx_gpio.o
 .debug_aranges
                0x000000d8       0x30 ./system/src/stm32f0-stdperiph/stm32f0xx_misc.o
 .debug_aranges
                0x00000108      0x160 ./system/src/stm32f0-stdperiph/stm32f0xx_rcc.o
 .debug_aranges
                0x00000268       0x58 ./system/src/stm32f0-stdperiph/stm32f0xx_syscfg.o
 .debug_aranges
                0x000002c0       0x28 ./system/src/newlib/_exit.o
 .debug_aranges
                0x000002e8       0x20 ./system/src/newlib/_sbrk.o
 .debug_aranges
                0x00000308       0x40 ./system/src/newlib/_startup.o
 .debug_aranges
                0x00000348       0x30 ./system/src/newlib/_syscalls.o
 .debug_aranges
                0x00000378       0x28 ./system/src/newlib/assert.o
 .debug_aranges
                0x000003a0       0x38 ./system/src/diag/Trace.o
 .debug_aranges
                0x000003d8       0x28 ./system/src/diag/trace_impl.o
 .debug_aranges
                0x00000400       0x28 ./system/src/cortexm/_initialize_hardware.o
 .debug_aranges
                0x00000428       0x58 ./system/src/cortexm/exception_handlers.o
 .debug_aranges
                0x00000480       0x30 ./system/src/cmsis/system_stm32f0xx.o
 .debug_aranges
                0x000004b0       0x20 ./system/src/cmsis/vectors_stm32f0xx.o
 .debug_aranges
                0x000004d0       0x20 ./src/main.o
 .debug_aranges
                0x000004f0       0x20 ./src/stm32f0xx_it.o

.debug_pubnames
 *(.debug_pubnames)

.debug_info     0x00000000     0x43fc
 *(.debug_info .gnu.linkonce.wi.*)
 .debug_info    0x00000000      0x437 ./system/src/stm32f0-stdperiph/stm32f0xx_exti.o
 .debug_info    0x00000437      0xa17 ./system/src/stm32f0-stdperiph/stm32f0xx_gpio.o
 .debug_info    0x00000e4e      0x406 ./system/src/stm32f0-stdperiph/stm32f0xx_misc.o
 .debug_info    0x00001254      0xf56 ./system/src/stm32f0-stdperiph/stm32f0xx_rcc.o
 .debug_info    0x000021aa      0x3d1 ./system/src/stm32f0-stdperiph/stm32f0xx_syscfg.o
 .debug_info    0x0000257b      0x100 ./system/src/newlib/_exit.o
 .debug_info    0x0000267b      0x125 ./system/src/newlib/_sbrk.o
 .debug_info    0x000027a0      0x474 ./system/src/newlib/_startup.o
 .debug_info    0x00002c14      0x1a9 ./system/src/newlib/_syscalls.o
 .debug_info    0x00002dbd      0x1b0 ./system/src/newlib/assert.o
 .debug_info    0x00002f6d      0x32b ./system/src/diag/Trace.o
 .debug_info    0x00003298       0xf8 ./system/src/diag/trace_impl.o
 .debug_info    0x00003390       0xc3 ./system/src/cortexm/_initialize_hardware.o
 .debug_info    0x00003453      0x335 ./system/src/cortexm/exception_handlers.o
 .debug_info    0x00003788      0x2e8 ./system/src/cmsis/system_stm32f0xx.o
 .debug_info    0x00003a70       0xd1 ./system/src/cmsis/vectors_stm32f0xx.o
 .debug_info    0x00003b41      0x5dd ./src/main.o
 .debug_info    0x0000411e      0x2de ./src/stm32f0xx_it.o

.debug_abbrev   0x00000000     0x167d
 *(.debug_abbrev)
 .debug_abbrev  0x00000000      0x1e6 ./system/src/stm32f0-stdperiph/stm32f0xx_exti.o
 .debug_abbrev  0x000001e6      0x1db ./system/src/stm32f0-stdperiph/stm32f0xx_gpio.o
 .debug_abbrev  0x000003c1      0x16e ./system/src/stm32f0-stdperiph/stm32f0xx_misc.o
 .debug_abbrev  0x0000052f      0x23e ./system/src/stm32f0-stdperiph/stm32f0xx_rcc.o
 .debug_abbrev  0x0000076d      0x195 ./system/src/stm32f0-stdperiph/stm32f0xx_syscfg.o
 .debug_abbrev  0x00000902       0xa4 ./system/src/newlib/_exit.o
 .debug_abbrev  0x000009a6       0xbb ./system/src/newlib/_sbrk.o
 .debug_abbrev  0x00000a61      0x1e9 ./system/src/newlib/_startup.o
 .debug_abbrev  0x00000c4a       0xe7 ./system/src/newlib/_syscalls.o
 .debug_abbrev  0x00000d31       0xc9 ./system/src/newlib/assert.o
 .debug_abbrev  0x00000dfa      0x178 ./system/src/diag/Trace.o
 .debug_abbrev  0x00000f72       0x9c ./system/src/diag/trace_impl.o
 .debug_abbrev  0x0000100e       0x63 ./system/src/cortexm/_initialize_hardware.o
 .debug_abbrev  0x00001071      0x165 ./system/src/cortexm/exception_handlers.o
 .debug_abbrev  0x000011d6      0x146 ./system/src/cmsis/system_stm32f0xx.o
 .debug_abbrev  0x0000131c       0x9d ./system/src/cmsis/vectors_stm32f0xx.o
 .debug_abbrev  0x000013b9      0x16d ./src/main.o
 .debug_abbrev  0x00001526      0x157 ./src/stm32f0xx_it.o

.debug_line     0x00000000     0x446d
 *(.debug_line)
 .debug_line    0x00000000      0x529 ./system/src/stm32f0-stdperiph/stm32f0xx_exti.o
 .debug_line    0x00000529      0x703 ./system/src/stm32f0-stdperiph/stm32f0xx_gpio.o
 .debug_line    0x00000c2c      0x389 ./system/src/stm32f0-stdperiph/stm32f0xx_misc.o
 .debug_line    0x00000fb5      0x9d0 ./system/src/stm32f0-stdperiph/stm32f0xx_rcc.o
 .debug_line    0x00001985      0x477 ./system/src/stm32f0-stdperiph/stm32f0xx_syscfg.o
 .debug_line    0x00001dfc      0x209 ./system/src/newlib/_exit.o
 .debug_line    0x00002005      0x1ab ./system/src/newlib/_sbrk.o
 .debug_line    0x000021b0      0x26a ./system/src/newlib/_startup.o
 .debug_line    0x0000241a      0x28d ./system/src/newlib/_syscalls.o
 .debug_line    0x000026a7      0x240 ./system/src/newlib/assert.o
 .debug_line    0x000028e7      0x265 ./system/src/diag/Trace.o
 .debug_line    0x00002b4c      0x47f ./system/src/diag/trace_impl.o
 .debug_line    0x00002fcb      0x345 ./system/src/cortexm/_initialize_hardware.o
 .debug_line    0x00003310      0x539 ./system/src/cortexm/exception_handlers.o
 .debug_line    0x00003849      0x383 ./system/src/cmsis/system_stm32f0xx.o
 .debug_line    0x00003bcc       0xd9 ./system/src/cmsis/vectors_stm32f0xx.o
 .debug_line    0x00003ca5      0x492 ./src/main.o
 .debug_line    0x00004137      0x336 ./src/stm32f0xx_it.o

.debug_frame    0x00000000      0xde4
 *(.debug_frame)
 .debug_frame   0x00000000       0xc0 ./system/src/stm32f0-stdperiph/stm32f0xx_exti.o
 .debug_frame   0x000000c0      0x168 ./system/src/stm32f0-stdperiph/stm32f0xx_gpio.o
 .debug_frame   0x00000228       0x60 ./system/src/stm32f0-stdperiph/stm32f0xx_misc.o
 .debug_frame   0x00000288      0x3f8 ./system/src/stm32f0-stdperiph/stm32f0xx_rcc.o
 .debug_frame   0x00000680       0xd4 ./system/src/stm32f0-stdperiph/stm32f0xx_syscfg.o
 .debug_frame   0x00000754       0x38 ./system/src/newlib/_exit.o
 .debug_frame   0x0000078c       0x28 ./system/src/newlib/_sbrk.o
 .debug_frame   0x000007b4       0x80 ./system/src/newlib/_startup.o
 .debug_frame   0x00000834       0x50 ./system/src/newlib/_syscalls.o
 .debug_frame   0x00000884       0x44 ./system/src/newlib/assert.o
 .debug_frame   0x000008c8       0x78 ./system/src/diag/Trace.o
 .debug_frame   0x00000940       0x30 ./system/src/diag/trace_impl.o
 .debug_frame   0x00000970       0x40 ./system/src/cortexm/_initialize_hardware.o
 .debug_frame   0x000009b0       0xb0 ./system/src/cortexm/exception_handlers.o
 .debug_frame   0x00000a60       0x54 ./system/src/cmsis/system_stm32f0xx.o
 .debug_frame   0x00000ab4       0x20 ./system/src/cmsis/vectors_stm32f0xx.o
 .debug_frame   0x00000ad4       0x30 ./src/main.o
 .debug_frame   0x00000b04       0x28 ./src/stm32f0xx_it.o
 .debug_frame   0x00000b2c       0x20 c:/arm/arm/bin/../lib/gcc/arm-none-eabi/4.9.3/armv6-m\libgcc.a(_udivsi3.o)
 .debug_frame   0x00000b4c       0x20 c:/arm/arm/bin/../lib/gcc/arm-none-eabi/4.9.3/../../../../arm-none-eabi/lib/armv6-m\libg_nano.a(lib_a-errno.o)
 .debug_frame   0x00000b6c       0x20 c:/arm/arm/bin/../lib/gcc/arm-none-eabi/4.9.3/../../../../arm-none-eabi/lib/armv6-m\libg_nano.a(lib_a-strlen.o)
 .debug_frame   0x00000b8c       0x4c c:/arm/arm/bin/../lib/gcc/arm-none-eabi/4.9.3/../../../../arm-none-eabi/lib/armv6-m\libg_nano.a(lib_a-vsnprintf.o)
 .debug_frame   0x00000bd8       0x74 c:/arm/arm/bin/../lib/gcc/arm-none-eabi/4.9.3/../../../../arm-none-eabi/lib/armv6-m\libg_nano.a(lib_a-nano-svfprintf.o)
 .debug_frame   0x00000c4c       0x54 c:/arm/arm/bin/../lib/gcc/arm-none-eabi/4.9.3/../../../../arm-none-eabi/lib/armv6-m\libg_nano.a(lib_a-nano-vfprintf_i.o)
 .debug_frame   0x00000ca0       0x20 c:/arm/arm/bin/../lib/gcc/arm-none-eabi/4.9.3/../../../../arm-none-eabi/lib/armv6-m\libg_nano.a(lib_a-memchr.o)
 .debug_frame   0x00000cc0       0x28 c:/arm/arm/bin/../lib/gcc/arm-none-eabi/4.9.3/../../../../arm-none-eabi/lib/armv6-m\libg_nano.a(lib_a-memcpy.o)
 .debug_frame   0x00000ce8       0x28 c:/arm/arm/bin/../lib/gcc/arm-none-eabi/4.9.3/../../../../arm-none-eabi/lib/armv6-m\libg_nano.a(lib_a-memmove.o)
 .debug_frame   0x00000d10       0x2c c:/arm/arm/bin/../lib/gcc/arm-none-eabi/4.9.3/../../../../arm-none-eabi/lib/armv6-m\libg_nano.a(lib_a-nano-freer.o)
 .debug_frame   0x00000d3c       0x2c c:/arm/arm/bin/../lib/gcc/arm-none-eabi/4.9.3/../../../../arm-none-eabi/lib/armv6-m\libg_nano.a(lib_a-nano-mallocr.o)
 .debug_frame   0x00000d68       0x30 c:/arm/arm/bin/../lib/gcc/arm-none-eabi/4.9.3/../../../../arm-none-eabi/lib/armv6-m\libg_nano.a(lib_a-nano-reallocr.o)
 .debug_frame   0x00000d98       0x2c c:/arm/arm/bin/../lib/gcc/arm-none-eabi/4.9.3/../../../../arm-none-eabi/lib/armv6-m\libg_nano.a(lib_a-sbrkr.o)
 .debug_frame   0x00000dc4       0x20 c:/arm/arm/bin/../lib/gcc/arm-none-eabi/4.9.3/../../../../arm-none-eabi/lib/armv6-m\libg_nano.a(lib_a-nano-msizer.o)

.debug_str      0x00000000    0x4571d
 *(.debug_str)
 .debug_str     0x00000000    0x3f0a2 ./system/src/stm32f0-stdperiph/stm32f0xx_exti.o
                              0x3f21f (size before relaxing)
 .debug_str     0x0003f0a2      0x2ec ./system/src/stm32f0-stdperiph/stm32f0xx_gpio.o
                              0x3f35a (size before relaxing)
 .debug_str     0x0003f38e      0x160 ./system/src/stm32f0-stdperiph/stm32f0xx_misc.o
                              0x3f1a9 (size before relaxing)
 .debug_str     0x0003f4ee      0x658 ./system/src/stm32f0-stdperiph/stm32f0xx_rcc.o
                              0x3f6f1 (size before relaxing)
 .debug_str     0x0003fb46      0x188 ./system/src/stm32f0-stdperiph/stm32f0xx_syscfg.o
                              0x3f1ce (size before relaxing)
 .debug_str     0x0003fcce     0x37d3 ./system/src/newlib/_exit.o
                               0x5cb0 (size before relaxing)
 .debug_str     0x000434a1      0x4de ./system/src/newlib/_sbrk.o
                               0x4422 (size before relaxing)
 .debug_str     0x0004397f      0x266 ./system/src/newlib/_startup.o
                               0x3ff8 (size before relaxing)
 .debug_str     0x00043be5      0xc2d ./system/src/newlib/_syscalls.o
                               0x5ed5 (size before relaxing)
 .debug_str     0x00044812       0xd5 ./system/src/newlib/assert.o
                               0x67b5 (size before relaxing)
 .debug_str     0x000448e7      0x9ac ./system/src/diag/Trace.o
                               0x65c1 (size before relaxing)
 .debug_str     0x00045293       0x50 ./system/src/diag/trace_impl.o
                              0x41b8a (size before relaxing)
 .debug_str     0x000452e3       0x4e ./system/src/cortexm/_initialize_hardware.o
                              0x3f077 (size before relaxing)
 .debug_str     0x00045331      0x13f ./system/src/cortexm/exception_handlers.o
                              0x428ae (size before relaxing)
 .debug_str     0x00045470       0x5e ./system/src/cmsis/system_stm32f0xx.o
                              0x3f125 (size before relaxing)
 .debug_str     0x000454ce       0x56 ./system/src/cmsis/vectors_stm32f0xx.o
                               0x2eee (size before relaxing)
 .debug_str     0x00045524      0x1be ./src/main.o
                              0x4346d (size before relaxing)
 .debug_str     0x000456e2       0x3b ./src/stm32f0xx_it.o
                              0x3f0fc (size before relaxing)

.debug_loc      0x00000000     0x1d72
 *(.debug_loc)
 .debug_loc     0x00000000      0x1a7 ./system/src/stm32f0-stdperiph/stm32f0xx_exti.o
 .debug_loc     0x000001a7      0x51a ./system/src/stm32f0-stdperiph/stm32f0xx_gpio.o
 .debug_loc     0x000006c1       0xdf ./system/src/stm32f0-stdperiph/stm32f0xx_misc.o
 .debug_loc     0x000007a0      0xc92 ./system/src/stm32f0-stdperiph/stm32f0xx_rcc.o
 .debug_loc     0x00001432      0x236 ./system/src/stm32f0-stdperiph/stm32f0xx_syscfg.o
 .debug_loc     0x00001668       0x7b ./system/src/newlib/_sbrk.o
 .debug_loc     0x000016e3      0x265 ./system/src/newlib/_startup.o
 .debug_loc     0x00001948       0x63 ./system/src/newlib/_syscalls.o
 .debug_loc     0x000019ab       0xf7 ./system/src/newlib/assert.o
 .debug_loc     0x00001aa2       0xf7 ./system/src/diag/Trace.o
 .debug_loc     0x00001b99       0x21 ./system/src/diag/trace_impl.o
 .debug_loc     0x00001bba       0x94 ./system/src/cortexm/exception_handlers.o
 .debug_loc     0x00001c4e       0xe2 ./system/src/cmsis/system_stm32f0xx.o
 .debug_loc     0x00001d30       0x42 ./src/main.o

.debug_macinfo
 *(.debug_macinfo)

.debug_weaknames
 *(.debug_weaknames)

.debug_funcnames
 *(.debug_funcnames)

.debug_typenames
 *(.debug_typenames)

.debug_varnames
 *(.debug_varnames)
OUTPUT(stm32f030_freq_div.elf elf32-littlearm)

.debug_ranges   0x00000000      0x408
 .debug_ranges  0x00000000       0x48 ./system/src/stm32f0-stdperiph/stm32f0xx_exti.o
 .debug_ranges  0x00000048       0x70 ./system/src/stm32f0-stdperiph/stm32f0xx_gpio.o
 .debug_ranges  0x000000b8       0x20 ./system/src/stm32f0-stdperiph/stm32f0xx_misc.o
 .debug_ranges  0x000000d8      0x150 ./system/src/stm32f0-stdperiph/stm32f0xx_rcc.o
 .debug_ranges  0x00000228       0x48 ./system/src/stm32f0-stdperiph/stm32f0xx_syscfg.o
 .debug_ranges  0x00000270       0x18 ./system/src/newlib/_exit.o
 .debug_ranges  0x00000288       0x10 ./system/src/newlib/_sbrk.o
 .debug_ranges  0x00000298       0x48 ./system/src/newlib/_startup.o
 .debug_ranges  0x000002e0       0x20 ./system/src/newlib/_syscalls.o
 .debug_ranges  0x00000300       0x18 ./system/src/newlib/assert.o
 .debug_ranges  0x00000318       0x28 ./system/src/diag/Trace.o
 .debug_ranges  0x00000340       0x18 ./system/src/diag/trace_impl.o
 .debug_ranges  0x00000358       0x18 ./system/src/cortexm/_initialize_hardware.o
 .debug_ranges  0x00000370       0x48 ./system/src/cortexm/exception_handlers.o
 .debug_ranges  0x000003b8       0x20 ./system/src/cmsis/system_stm32f0xx.o
 .debug_ranges  0x000003d8       0x10 ./system/src/cmsis/vectors_stm32f0xx.o
 .debug_ranges  0x000003e8       0x10 ./src/main.o
 .debug_ranges  0x000003f8       0x10 ./src/stm32f0xx_it.o

.debug_macro    0x00000000     0xd0cd
 .debug_macro   0x00000000      0x15c ./system/src/stm32f0-stdperiph/stm32f0xx_exti.o
 .debug_macro   0x0000015c      0x844 ./system/src/stm32f0-stdperiph/stm32f0xx_exti.o
 .debug_macro   0x000009a0       0x7a ./system/src/stm32f0-stdperiph/stm32f0xx_exti.o
 .debug_macro   0x00000a1a       0x3a ./system/src/stm32f0-stdperiph/stm32f0xx_exti.o
 .debug_macro   0x00000a54      0x34e ./system/src/stm32f0-stdperiph/stm32f0xx_exti.o
 .debug_macro   0x00000da2       0x1f ./system/src/stm32f0-stdperiph/stm32f0xx_exti.o
 .debug_macro   0x00000dc1      0x242 ./system/src/stm32f0-stdperiph/stm32f0xx_exti.o
 .debug_macro   0x00001003     0x5b9e ./system/src/stm32f0-stdperiph/stm32f0xx_exti.o
 .debug_macro   0x00006ba1      0x2ec ./system/src/stm32f0-stdperiph/stm32f0xx_exti.o
 .debug_macro   0x00006e8d      0x3cf ./system/src/stm32f0-stdperiph/stm32f0xx_exti.o
 .debug_macro   0x0000725c      0x191 ./system/src/stm32f0-stdperiph/stm32f0xx_exti.o
 .debug_macro   0x000073ed       0x46 ./system/src/stm32f0-stdperiph/stm32f0xx_exti.o
 .debug_macro   0x00007433       0xd9 ./system/src/stm32f0-stdperiph/stm32f0xx_exti.o
 .debug_macro   0x0000750c       0xef ./system/src/stm32f0-stdperiph/stm32f0xx_exti.o
 .debug_macro   0x000075fb      0x184 ./system/src/stm32f0-stdperiph/stm32f0xx_exti.o
 .debug_macro   0x0000777f       0x7c ./system/src/stm32f0-stdperiph/stm32f0xx_exti.o
 .debug_macro   0x000077fb      0x295 ./system/src/stm32f0-stdperiph/stm32f0xx_exti.o
 .debug_macro   0x00007a90      0x23d ./system/src/stm32f0-stdperiph/stm32f0xx_exti.o
 .debug_macro   0x00007ccd      0x185 ./system/src/stm32f0-stdperiph/stm32f0xx_exti.o
 .debug_macro   0x00007e52      0x184 ./system/src/stm32f0-stdperiph/stm32f0xx_exti.o
 .debug_macro   0x00007fd6      0x2a0 ./system/src/stm32f0-stdperiph/stm32f0xx_exti.o
 .debug_macro   0x00008276       0x70 ./system/src/stm32f0-stdperiph/stm32f0xx_exti.o
 .debug_macro   0x000082e6       0xdf ./system/src/stm32f0-stdperiph/stm32f0xx_exti.o
 .debug_macro   0x000083c5      0x522 ./system/src/stm32f0-stdperiph/stm32f0xx_exti.o
 .debug_macro   0x000088e7      0x4c5 ./system/src/stm32f0-stdperiph/stm32f0xx_exti.o
 .debug_macro   0x00008dac      0x397 ./system/src/stm32f0-stdperiph/stm32f0xx_exti.o
 .debug_macro   0x00009143      0x750 ./system/src/stm32f0-stdperiph/stm32f0xx_exti.o
 .debug_macro   0x00009893      0x353 ./system/src/stm32f0-stdperiph/stm32f0xx_exti.o
 .debug_macro   0x00009be6       0x34 ./system/src/stm32f0-stdperiph/stm32f0xx_exti.o
 .debug_macro   0x00009c1a       0x3a ./system/src/stm32f0-stdperiph/stm32f0xx_exti.o
 .debug_macro   0x00009c54       0xd1 ./system/src/stm32f0-stdperiph/stm32f0xx_exti.o
 .debug_macro   0x00009d25      0x156 ./system/src/stm32f0-stdperiph/stm32f0xx_gpio.o
 .debug_macro   0x00009e7b       0xd7 ./system/src/stm32f0-stdperiph/stm32f0xx_gpio.o
 .debug_macro   0x00009f52      0x17f ./system/src/stm32f0-stdperiph/stm32f0xx_gpio.o
 .debug_macro   0x0000a0d1      0x156 ./system/src/stm32f0-stdperiph/stm32f0xx_misc.o
 .debug_macro   0x0000a227       0x34 ./system/src/stm32f0-stdperiph/stm32f0xx_misc.o
 .debug_macro   0x0000a25b      0x174 ./system/src/stm32f0-stdperiph/stm32f0xx_rcc.o
 .debug_macro   0x0000a3cf      0x51c ./system/src/stm32f0-stdperiph/stm32f0xx_rcc.o
 .debug_macro   0x0000a8eb      0x156 ./system/src/stm32f0-stdperiph/stm32f0xx_syscfg.o
 .debug_macro   0x0000aa41      0x17e ./system/src/stm32f0-stdperiph/stm32f0xx_syscfg.o
 .debug_macro   0x0000abbf      0x128 ./system/src/newlib/_exit.o
 .debug_macro   0x0000ace7       0x9c ./system/src/newlib/_exit.o
 .debug_macro   0x0000ad83      0x10e ./system/src/newlib/_exit.o
 .debug_macro   0x0000ae91       0x86 ./system/src/newlib/_exit.o
 .debug_macro   0x0000af17       0x43 ./system/src/newlib/_exit.o
 .debug_macro   0x0000af5a      0x27a ./system/src/newlib/_exit.o
 .debug_macro   0x0000b1d4       0x35 ./system/src/newlib/_exit.o
 .debug_macro   0x0000b209       0xd1 ./system/src/newlib/_sbrk.o
 .debug_macro   0x0000b2da       0x19 ./system/src/newlib/_sbrk.o
 .debug_macro   0x0000b2f3      0x16d ./system/src/newlib/_sbrk.o
 .debug_macro   0x0000b460       0x10 ./system/src/newlib/_sbrk.o
 .debug_macro   0x0000b470      0x23b ./system/src/newlib/_sbrk.o
 .debug_macro   0x0000b6ab       0xdb ./system/src/newlib/_startup.o
 .debug_macro   0x0000b786      0x17c ./system/src/newlib/_syscalls.o
 .debug_macro   0x0000b902       0x1c ./system/src/newlib/_syscalls.o
 .debug_macro   0x0000b91e       0x10 ./system/src/newlib/_syscalls.o
 .debug_macro   0x0000b92e       0x10 ./system/src/newlib/_syscalls.o
 .debug_macro   0x0000b93e       0x10 ./system/src/newlib/_syscalls.o
 .debug_macro   0x0000b94e       0x35 ./system/src/newlib/_syscalls.o
 .debug_macro   0x0000b983      0x121 ./system/src/newlib/_syscalls.o
 .debug_macro   0x0000baa4       0x22 ./system/src/newlib/_syscalls.o
 .debug_macro   0x0000bac6       0x2b ./system/src/newlib/_syscalls.o
 .debug_macro   0x0000baf1      0x118 ./system/src/newlib/_syscalls.o
 .debug_macro   0x0000bc09      0x13e ./system/src/newlib/_syscalls.o
 .debug_macro   0x0000bd47       0x16 ./system/src/newlib/_syscalls.o
 .debug_macro   0x0000bd5d      0x144 ./system/src/newlib/assert.o
 .debug_macro   0x0000bea1       0x1c ./system/src/newlib/assert.o
 .debug_macro   0x0000bebd      0x14f ./system/src/diag/Trace.o
 .debug_macro   0x0000c00c       0x16 ./system/src/diag/Trace.o
 .debug_macro   0x0000c022       0x97 ./system/src/diag/Trace.o
 .debug_macro   0x0000c0b9       0xf6 ./system/src/diag/Trace.o
 .debug_macro   0x0000c1af       0x10 ./system/src/diag/Trace.o
 .debug_macro   0x0000c1bf       0x16 ./system/src/diag/Trace.o
 .debug_macro   0x0000c1d5      0x196 ./system/src/diag/Trace.o
 .debug_macro   0x0000c36b       0x52 ./system/src/diag/Trace.o
 .debug_macro   0x0000c3bd       0x16 ./system/src/diag/Trace.o
 .debug_macro   0x0000c3d3      0x22f ./system/src/diag/trace_impl.o
 .debug_macro   0x0000c602       0x10 ./system/src/diag/trace_impl.o
 .debug_macro   0x0000c612       0xc8 ./system/src/diag/trace_impl.o
 .debug_macro   0x0000c6da       0xbe ./system/src/diag/trace_impl.o
 .debug_macro   0x0000c798      0x156 ./system/src/cortexm/_initialize_hardware.o
 .debug_macro   0x0000c8ee      0x275 ./system/src/cortexm/exception_handlers.o
 .debug_macro   0x0000cb63       0x22 ./system/src/cortexm/exception_handlers.o
 .debug_macro   0x0000cb85       0x10 ./system/src/cortexm/exception_handlers.o
 .debug_macro   0x0000cb95      0x14c ./system/src/cmsis/system_stm32f0xx.o
 .debug_macro   0x0000cce1       0x2e ./system/src/cmsis/vectors_stm32f0xx.o
 .debug_macro   0x0000cd0f      0x264 ./src/main.o
 .debug_macro   0x0000cf73      0x15a ./src/stm32f0xx_it.o
